:020000001F29B6
:080008000428831287138316FC
:1000100087178312080083128713831687138312AE
:100020000800831207178316071383120800831230
:10003000071383160713831208000630B500B50BAB
:100040001F2808001030B500B50B1F280800FF302E
:1000500087000030831687008312080011202220B9
:100060000B202220172022202220222008002220DC
:10007000172022200B2022201120222005202220C0
:1000800008001720222005202220112022200B20EA
:100090002220172022200800172022200B202220B7
:1000A00011202220172022200520222008001720BE
:1000B0002220052022201120222017202220222069
:1000C00008002220172022200B202220112040305F
:1000D000B500B50B692805204030B500B50B6E287A
:1000E0001720222011202220172022201120222038
:1000F0001720222011202220172022201120222028
:100100001720222011202220172022201120222017
:100110001720222011202220172022201120222007
:100120001720222011202220080083121D203308CE
:10013000320503199D2805209F280B209F28831234
:100140001D201120222017200800B2008030B300AB
:1001500095200310B30CB308031DA8281D2005200B
:100160001D2011201D2007088039803AB4001D2071
:1001700017201D200800B2000830B300952003109E
:10018000B30CB308031DBE281D2005201D2011201F
:100190001D2007088039803AB4001D2017201D203B
:1001A0000800831205201720222011201D20070897
:1001B00080390319DD283308B2041D2017200800F8
:1001C0000030B2008030B300D1200310B30CB3086C
:1001D000031DE42832080800831288008316880172
:1001E00083120514FF301621FF3016210510FF3051
:1001F0001621FF301621F12808008312880083168B
:1002000088018312051430300A21051003300A21B9
:1002100002290800B500FF30B600FF30B700B70B69
:100220000F29B60B0D29B50B0B290800B500FF30BF
:10023000B600B60B1929B50B172908001E2927206F
:100240006120831285018801831606309F002030CB
:100250008500880183128501B001B101851E5229F4
:100260002E20A630A5200130B4080319EC20300858
:10027000A5200230B4080319EC203108A520033072
:10028000B4080319EC2037202E20A630A520043016
:10029000B40803194429B00AB10A301E30293720A6
:1002A000103016212E20A630A5200530B4080319E1
:1002B000EC20B0013008A5200630B4080319EC206A
:1002C00037202E20A730A5200730B4080319EC20D2
:1002D00085140000000000008510E0203008320284
:1002E0000830031DEC20B00A301A78294C206D2903
:0602F000572037201E21FB
:00000001FF
